:030000000219FDE5
:03000B000200AA46
:03002B0002015C73
:03005B000202EBB3
:030073000202D8AE
:1000800002030406080C10182030406080040608A3
:100090000C10182030406080A0C00003070F1F0D17
:1000A0000D0403060D0503030202C2AFC0D0C0E079
:1000B000206214E5256009E473E525F4F58AD2622F
:1000C000D0E0D0D0D2AF3285268AC262E526F46075
:1000D0002F30682520720DD0E0D0D0C2B1C287C2C7
:1000E00081D2AF32C2B1C287C281206F0C206609B3
:1000F000740AD5E0FDE57B4280D0E0D0D0D2AF32AB
:10010000758A00C28DD26201F901B9306805206696
:1001100002D2B101B9306805206602D28701B93038
:100120006805206602D28101B9C28230680A206661
:10013000077408D5E0FDD2B101B9C28630680A2043
:1001400066077408D5E0FDD28701B9C28030680A1D
:100150002066077408D5E0FDD28101B9C2AFC2ADF7
:1001600053E6EFC0D0C0E0D2D3D2AFC2CEE52A6012
:1001700007207449152A21BD7800790020742EE5E6
:1001800080307E01F430E50278FF53DACF207E0321
:1001900043DA20307E0343DA10C2D8C271E58030E2
:1001A0007E01F430E50279FFC3E89970CB3061033A
:1001B000752A40207403752A40885CD27020740D23
:1001C000E52B6004152B21CD43DA01C2D820700243
:1001D00021E0A85C206102C27020740221DE882226
:1001E0007882B60403852224C3E52594404002D2D8
:1001F0006420CF0AD0E0D0D043E610D2AD32C2CFD7
:10020000053A7802E52A6005307402152AC3E55CD8
:1002100094014005755F00412A756000756900E52D
:100220005F2401F55F5003755FFF7982B7020D30DF
:100230006E1DC3E52294324016854C227982B703A5
:100240000E306E0BC3E52294324004798E8722C3B0
:10025000E5239522600840041523415E0523D8CA92
:100260000569E56970021569D56A63756A017805E3
:10027000C3E569956B4057C3E569956C50087801F3
:10028000756A03020292C3E569956D5005780175A0
:100290006A01C3E5629524401E7982B7040241C316
:1002A000206E14852462E569046003856B69756AB4
:1002B0000175233C0202CEE5622850057562FF41BC
:1002C000C3F562E5620470067560FF7569FFD0E0F2
:1002D000D0D043E610D2AD32C2AF53E67F7592FA6A
:1002E0007593FFC260759104D2AF32C2AF53E6EF8F
:1002F000C2ADC0D0C0E0C0F0D2D3D2AFA8FBA9FC41
:10030000C2D8307102615253DACF207E0343DA1033
:10031000307E0343DA20D271E580307E01F420E59F
:1003200002612988278928A13753DACF207E034329
:10033000DA20307E0343DA10C2D8C271307402A1D1
:10034000237800E580307E01F430E502A123885C4B
:10035000A10B53DACF207E0343DA20307E0343DA49
:1003600010C271206102812B53DACF207E0343DA61
:1003700010307E0343DA20C2D8D27188578958C31F
:10038000E89555F8E99556F97B007E087A00C3E8B0
:10039000948CE994005005755B00811D882178A23A
:1003A000E6A8216055C3E894C8E994005008E4D257
:1003B000E4FB7A0A61F8C3E89468E994015008E420
:1003C000D2E3FB7A0F61F8C3E894D0E994025008B5
:1003D000E4D2E2FB7A1E61F8C3E894A0E9940550E8
:1003E00008E4D2E1FB7A3C61F8C3E89498E9940808
:1003F0005008E4D2E0FB7A787E00C3E89559FCE926
:10040000955AFD30E70AECF42401FCEDF43400FDCC
:10041000755B00C3EC9AED9E5003755B01885989AA
:100420005A8557558558567802A10BC3E89527F889
:10043000E99528F9307C0281EF307B0281EF307A38
:100440000281E8207502814EE9FDE8FC816DE9C377
:1004500013F9E813F830790281E8E9C313F9E813D6
:10046000F830780281E8E9C313FDE813FC20612C21
:0F047000C3EC941CED940240028184ED701EC316
:10047F00EC94C850180529E52970021529C3E52900
:10048F00940A5002A123755C00D270A123E5296064
:10049F000215297400207F037896E624FAFEE434CF
:1004AF0000FFC3EC9EFCED9FFD50067800790081A4
:1004BF00EFC3EC94FFED9400400678FF790081EFD5
:1004CF00EC8572F0A4C5F0A2F733F879004003026F
:1004DF00050B78FF790002050BE9C313F9E813F850
:1004EF00307C0EE9600278FFC3E81338F8E434007B
:1004FF00F9C3E894FFE99400400278FF885CD2705A
:10050F00206102A123741FF4552F4BF52FC274EBFA
:10051F007002D274752A40307403752A0A30610252
:10052F00A13720740353DAFE207403752B20D0F00B
:10053F00D0E0D0D0D2AD43E6103279010205677911
:10054F0003020567790A020567791E020567796458
:10055F0002056779C80205677817E4D5E0FDD8FA78
:10056F00D9F6227A147B7802058E7A107B8C0205DD
:10057F008E7A0D7BB402058E7A0B7BC802058E79BD
:10058F0002E4C286D5E0FDD287D5E0FDC287D5E073
:10059F00FDD286D5E0FDE920E002D2B130E002D2F3
:1005AF0081E573D5E0FDE920E002C2B130E002C27F
:1005BF00817496D5E0FDD9C9EAF8D5E0FDD8FBDB0B
:1005CF00BEC28622C37C007D0075F00005F0EA33C1
:1005DF00FAEB33FB50F6EB13FBEA13FAC3E9FFE830
:1005EF00FEE89AF8E99BF95004EFF9EEF8B3EC3313
:1005FF00FCED33FDD5F0DFEDF9ECF822E889F08A58
:10060F0020D2D4F8A9F07B0030F70B7BFFF4240144
:10061F00F8E9F43400F9E88520F0A4ADF0F8E985A5
:10062F0020F0A4AFF0FEED2EF974003FFA7C04C366
:10063F00EA13FAE913F9E813F8DCF48BF030F70A50
:10064F00E8F42401F8E9F43400F9E889F0C2D4F8A9
:10065F00A9F0227882B60403020701C3E55C94195E
:10066F00401EE52D54067018206E3678057994E7F4
:10067F00146007780A1460027812C3E54198401F8E
:10068F00306E098564627569FF756A01852224E4FD
:10069F00F544F545F546F547F548C26E020701D218
:1006AF006E7994E7147013E523F43333F913F8E9F3
:1006BF00540104F9E854FE0206F5E714147014E52A
:1006CF0023F4333333F913F8E9540304F9E854FCF2
:1006DF000206FDE523F433333333F913F8E95407F6
:1006EF000404F9E854F8C39440F8E99400F98844F5
:1006FF00894522C3E54113F9E54013F8C3E5449852
:10070F00F8E54599F9500CC3E89480E994FF401639
:10071F00020739C3E8947FE9940050030207397840
:10072F007F7900020739788079FF8849894A22E565
:10073F00492546F8E54A3547F9854A20E43007014F
:10074F00F43548FA30E709C3EA94F0401502077709
:10075F00C3EA940F500302077778FF79FF7A0F02ED
:10076F000777780079007AF0C3E5249561500AC3C2
:10077F0074019524500B020795E54A20E70E0207F6
:10078F0095E54A30E706884689478A482278A5E6E4
:10079F00FAC3E54933F8E54A33F9D10BE930E70BF2
:1007AF00C3E89480E994FF4013E1CFC3E8947FE955
:1007BF0094005002E1CF787F7900E1CF788079FF04
:1007CF00E820E715C3E52398F84009C3E8940140F2
:1007DF00030207F678010207F6E8F424012523F84F
:1007EF0040030207F678FF884B2278A6E6FAA8475F
:1007FF00A94812060BE930E70CC3E89401E994FF0E
:10080F00401602082BC3E894FFE994005003020836
:10081F002B78FF790002082B780179FFE920E71583
:10082F00C3E54B98F84009C3E8940140030208520E
:10083F007801020852E8F42401254BF8400302081E
:10084F005278FF88242278FFC26420693D206A1203
:10085F00D264C3E541940A4009C3E5259440500290
:0D086F00C26479A1E76023E541601F74FFBA
:10087C008541F0848539F0306A0375F005A4F8C51C
:10088C00F0600278FFC3E895645002A86488632284
:10089C00C3E5409440E5419401E56350031401AD78
:1008AC00046002F563227883E6F520120F2975E8BF
:1008BC009012054975E890E5E820ECFBA8BDA9BEAF
:1008CC00120FCF756E55756F00C3740013FD745500
:1008DC00606613FC74552CFC74003DFDECFAEDFBCA
:1008EC00C3E89AE99B4014E56E2455F56EE56F3428
:1008FC0000F56FEA2CFAEB3DFB80E5AE6EAF6FC3F3
:10090C00E56F13F9E56E13F8C3E913F9E813F87AF8
:10091C0003C3E913F9E813F8DAF7AA201A7009757A
:10092C006E00756F000209441AEA6008EE28FEEFAB
:10093C0039FFDAF88E6E8F6F2275E890227883E695
:10094C00FFE5E820ECF7A8BDA9BE0570C3E57094DF
:10095C00084052757000E9FA79A0E76044EA700724
:10096C00E571601B02097FC3E895716010E5715059
:10097C0006600C1402098B0460F902098BE571F511
:10098C0071C394A8401B7561C0C394054013756175
:10099C0080C39405400B756140C394054003756199
:1009AC000075BB0622EFC39401601F7455601BC316
:1009BC00E894FFE994035012C3E8956EE9956F50E3
:1009CC0009E561600C15610209DDE561F460020561
:1009DC0061A861C3E524985002A824C3E89562403D
:1009EC000AA862E562F4600385626188258826E5C1
:1009FC0070B4070375BB1E22743279A787F0A4C5A7
:100A0C00F0A2F733F8C3E895614002A86188228808
:100A1C0024882588268864227540007541F022C2FE
:100A2C00AF75C820A8CCA9CDAA3A30CF010A75C899
:100A3C0024D2AFAB3BAC3C883B893CC3E89BF8E988
:100A4C009C206908F930670261374194AD3D8A3DBD
:100A5C00F9EA9DFA600478FF79FFAE3EAF3F8B3E1A
:100A6C008C3FA83BA93CC3E89EF8E99FF9C3E5413C
:100A7C0013FBE54013FAE82AF540E93BF541500633
:100A8C007540FF7541FF41DEAA40AB41AC40AD4122
:100A9C007E047F02C3EB940440021E1FC3EB940838
:100AAC0040021E1FC3ED13FDEC13FCDEF7C3EA9CE2
:100ABC00FAEB9DFBEF6009C3E913F9E813F8DFF7D4
:100ACC00EA28FAEB39FB8A408B4150067BFF8B40BE
:100ADC008B41C3EB94025002D2673069047F0361EF
:100AEC00097892E6FFC3E537948240110FC3E537CE
:100AFC0094A040010FC3EF940640027F057E02E5EF
:100B0C0041C4540FF9E541C454F0F8E540C4540F06
:100B1C0028F8C3E89EFAE99400FB4009C3EA940262
:100B2C00EB940050047A02E4FB6183AA40AB41EBE6
:100B3C00C4FEEAC4540F4EFCC3EA9CFAEB9400FBCF
:100B4C00C3E813C313F8EA28FAEB3400FB8A408B92
:100B5C0041C3EB94024002C2677802EBC4FE7B00F7
:100B6C00EAC4540F4EFAC3EA98FA4005C3940250F3
:100B7C00027A027892E6FF30600261838551928599
:100B8C005293D26043E680C3E49AF8E49BF9306751
:100B9C0002810FE8FAE9FBD3E913FDE813FC885155
:100BAC008952C3EF94036038EF20E00DE82CF8E98C
:100BBC003DF9ECFAEDFB020BD8E828F8E939F9C35A
:100BCC00E82402F8E93400F97AFE7BFFC3EF9403C2
:100BDC00400E8A538B54884D894E8C4F8D508143D7
:100BEC00885389548A4D8B4E8C4F8D5030691275B9
:100BFC0053F07554FF754FF07550FF7551F07552E9
:100C0C00FF8143E8FAD3E813FC8851C3EF940360E7
:100C1C0020EF20E007E82CF8ECFA812FE8282402DA
:100C2C00F87AFEC3EF940340088A53884D8C4F81A9
:100C3C004388538A4D8C4FE568C3335002646BF57F
:100C4C0068306002814D753402D26043E680E52D38
:100C5C0054066034A840A941C3E913F9E813F8C35A
:0F0C6C00E913F9E813F8306904E92440F9C2AF3D
:100C7B0053E67F759100C3E498F594E499F5957567
:100C8B009104D26043E680D2AF22D26575430075E2
:100C9B002000306C03752040020CB4D26575430004
:100CAB00752040306C037520007801790120672096
:100CBB00E52D54066002C2657914E541C31370013A
:100CCB0004F8C3941440027814306904781B791B20
:100CDB00206010E543600C306903D53404D26DA15C
:100CEB005691550543E59B5440B52002A140306910
:100CFB000908C3E89940011881DB20650A08C3E89D
:100D0B0099400281B481DBC265C2AF53E67F759116
:100D1B00003067127594007595FE759104D260438F
:100D2B00E680D2AF81B4AE40AF41C3E49EF594E40C
:100D3B009FF595A125C3E5339401500281B430652D
:100D4B000281B4D802A15481DBC26DC2AF53E67FDE
:100D5B00759100855394855495759104854D9285B5
:100D6B004E93D26043E680D2AFE52D540660082047
:100D7B006A020533020D92306D0D206C0A20650757
:100D8B001581158102162222780030640530650228
:100D9B007801E53775F007A4F9E5F028F5F0E9A23D
:100DAB00F013A2F113A2F213F537C3947850037525
:100DBB003778C3E53795384008D266C2B1C287C2CF
:100DCB0081306002A1CC854F92855093D26043E66F
:100DDB008022207D16C2AF754202C286D28230625B
:100DEB0002D281D2AF759F02020FCCC2AF75420205
:100DFB00C286D280306202D2B1D2AF759F02020F8F
:100E0B00CC307243207D20C2AF75420390013A75FE
:100E1B007B40C281C280306204D287C12AD286D283
:100E2B00AF759F03020FCCC2AF75420390013A75A9
:100E3B007B40C2B1C282306204D287C14AD286D211
:100E4B00AF759F01020FCC207D17C2AF7542039087
:100E5B000115C281306202D287D2AF759F03020F98
:100E6B00CCC2AF754203900115C2B1306202D2877A
:100E7B00D2AF759F01020FCC207D16C2AF75420415
:100E8B00C282D280306202D287D2AF759F01020F2D
:100E9B00CCC2AF754204C280D282306202D287D2FA
:100EAB00AF759F03020FCC307243207D20C2AF750C
:100EBB004205900129757B04C287C286306204D239
:100ECB00B1C1D0D282D2AF759F02020FCCC2AF7527
:100EDB00420590014B757B01C287C286306204D2FA
:100EEB0081C1F0D280D2AF759F02020FCC207D174B
:100EFB00C2AF75420590010BC287306202D2B1D2EC
:100F0B00AF759F02020FCCC2AF75420590011FC295
:100F1B00873062EBD281D2AF759F02020FCC207D5E
:100F2B0016C2AF754206C280D286306202D2B1D2EF
:100F3B00AF759F03020FCCC2AF754206C282D28639
:100F4B00306202D281D2AF759F01020FCC30724357
:100F5B00207D20C2AF75420190014B757B01C2B160
:100F6B00C282306204D281E176D280D2AF759F010A
:100F7B00020FCCC2AF754201900129757B04C2816F
:100F8B00C280306204D2B1E196D282D2AF759F0398
:100F9B00020FCC207D17C2AF75420190011FC2B169
:100FAB00306202D281D2AF759F01020FCCC2AF75F6
:100FBB00420190010BC281306202D2B1D2AF759F58
:100FCB0003C26622900109757B00C2B1C287C28140
:100FDB00C282C286C280C2622278807607087607F8
:100FEB000876010876040876FF0876FF087609086C
:100FFB007602087601087601788C7601087600086F
:10100B0076B40876FF0876FF0876FF087603087635
:10101B00FF0876010876FF0876250876D0087678E3
:10102B000876C80876040876FF087601087600086B
:10103B00767A08760A087601087601087600087633
:10104B00FF087600227887E6FFC272BF0302D272D6
:10105B007888C27DE630E102D27DC27E7889E630A7
:0F106B00E102D27EC3EF94026008758E01D2734A
:10107A00021082758E00C273227880E61490008076
:10108A009378A5F67881E6149000809378A6F6788E
:10109A0086E61490008D9378A7F6789FE6F870019B
:1010AA0008C3E8941140027811E82828F56B256BEB
:1010BA00256B28F56C256B2828F56D7886E6F539B9
:1010CA00C394025003753902789CE67538FFB4025E
:1010DA00037538A0B4030375388278A3E614900028
:1010EA009A93F566120FCF22C2B3789DE66002D2B8
:1010FA00B3227896E6FA7897E6FB7888E6B4030591
:10110A00C3EB940EFB307F047A007BFFC3EB9AFC9F
:10111A00C3948250027C827572000572EC8572F06B
:10112A00A4C3E5F0947D40F222D27F11FC12055847
:10113A007A007B007C1012054EE55C2AFA74003BAB
:10114A00FBDCF37C04C3EB13FBEA13FADCF7FEC205
:10115A007F11FC22E5EF20E6037520000520903D73
:10116A00FFE520146006901FFF14600093046003DB
:10117A0075EF1253D9BF7581C043FF8012054975B7
:10118A00EF0243B203E5B3240220E70DF521E5B1EE
:10119A0020E0068521B343B101120FCF758038755F
:1011AA00A4C775F1FF75D4DF7590FF75A50075F2B8
:1011BA000075D50075A0FF75A60075F30075D600F9
:1011CA0075B0E475A71B75F4FF75E241120FCFE401
:1011DA00F8F6D8FD756801120FE412167978988628
:1011EA0073753001C2AF12056212057212055812E8
:1011FA00057912055812058012055812179C120516
:10120A006212056212055DC2AF78FA79FA30850773
:10121A00D9FBD8F7021C001150118311F211FC7886
:10122A00988673120FCF75881075890275C8247550
:10123A00910475D84075A82275B80275E690759B19
:10124A0080759D0075D10E75BC5875BB0675BA1FA1
:10125A0075E880120549D2AF1208B275360053DA22
:10126A00CF207E0343DA20307E0343DA1043DA01CB
:10127A00C2D8C271120562D2617B037A0CE55B7037
:10128A00077A0CDB030212111205582070030212AE
:10129A0011C270E55CC3940240E1E52F541F855EDC
:1012AA005DF55EB55DD5DAD5C26153DACF207E032E
:1012BA0043DA20307E0343DA10C2D8C27178A2E63C
:1012CA007008D274E52F54E0F52FC2757529001203
:1012DA00055D307409C3E529940A4002D2751205E6
:1012EA004E78023074027800C3E55C9840F0C2AFD1
:1012FA00120572120572120572D2AF120562754C8E
:10130A000012054E788CE6C3940150030213E1E5FE
:10131A0030C3940150030213E1207435C3E55C9491
:10132A00FF50030213E1C2AF120587D2AF12055D67
:10133A00C3E55C940150EFC2AF1205721205531255
:10134A000572D2AF12055DC3E55C94FF40E902184D
:10135A00217F05D27F11FC12055DC2AFC27F11FC4D
:10136A00AE5CC3E55C947FD2AF4076120549C2AF4A
:10137A00120587D2AFDFDC3133C3EE94057897F6D6
:10138A001205621216BB1217A47F0AD27F11FC1231
:10139A00055DC2AFC27F11FCAE5CC3E55C947FD22F
:1013AA00AF50E6120549C2AF120572120553120573
:1013BA0072D2AFDFD63133EE24037896F612056285
:1013CA001216BB1217D312055D11FCC3E55C94FF1C
:1013DA0050026123021821C3E55C954C4003855CE9
:1013EA004C12055D78017988E7B403027805C3E5F4
:1013FA005C984002610BC2AF12058712058712057D
:10140A0087D2AF120562753000E4F531F532053145
:10141A00E531F4703F0532789AE67819146012784B
:10142A003214600D787D14600878FA1460037532FE
:10143A0000C3E53298401D120FCF120549153275C7
:10144A00310078998673C2AF120587D2AF78988631
:10145A007312055D120553E52A70053074024111B5
:0D146A0078012074027806C3E55C9840A16B
:1014770012055DE52A7003021211C2AF120FCFE405
:10148700F522F523F524F525F526F567D2AF7885FE
:10149700E6C333F565E4F544F545F546F547F54804
:1014A700F570F52CF52DF53775700875BB1E12050F
:1014B70049120945E5E820ECFBA8BDA9BEE9700182
:1014C700F8887112094975700875BB1E1150C2AFB3
:1014D7007561FF120A04852261852262852263D223
:1014E700AF7522017524017525017526018560698F
:1014F700756A017888E6B40307C27D307602D27D2B
:10150700D268D269753300120F29120F58120A24B4
:10151700120A2B120A24120A2B120A24120CA612E0
:101527000662120D93120DDD120A2B120C95306E06
:101537000312070220670312085530670312089C3D
:10154700120D93120E0C120A2B120CA6306E0312F8
:10155700073E120D93120E83120A2B120C95306E52
:101567000312079C120D93120EB2120A2B120CA62D
:10157700306E031207F9120D93120F29120A2B125C
:101587000945120C95120D93120F58120949120AA8
:101597002B30692C856461856462856069756A0191
:1015A70079187A0CC3E533994009C269D26A8A353A
:1015B7000215C7C3E55C9401400302152302162AEE
:1015C700306A1D206C1AE535147006C26AD26BA109
:1015D70023F535C3E55C9401400302152302162A5F
:1015E700753600C3E55F94014009856462856069CB
:1015F700756A0178FA79A4E760027803C3E55F9812
:101607005021307404E52A601A78F0306C0585643F
:10161700617820C3E541985002A1230536E55C6057
:1016270002C12D753600C2AF120FCF7887E6FE765E
:101637000211507887EEF6E4F522F523F524F52517
:10164700F526F565752C00752D00D2AF12055D12D4
:101657000FCF78A4E66006D2B1D287D28130740664
:10166700E52A70024111788DE6C39401400241E8F2
:101677008113901A0D78201216FDE520B4A50CA34E
:101687001216FDE520B45A0302169B120FE4121638
:10169700BB0216BA901A0378807B0A1216FDA308BC
:1016A700DBF9901A0F788C7B191216FDA308DBF96A
:1016B700901A2822C2AF12173C121716901A0074FC
:1016C7000E121702A37406121702A374151217023B
:1016D700901A0378807B0A121701A308DBF9901A86
:1016E7000F788C7B19121701A308DBF912174F1219
:1016F700172D901A2822E493F622E6438F01538F81
:10170700FD75EF0275B7A575B7F1F0538FFE22434C
:101717008F02438F0175EF0275B7A575B7F1901A60
:101727000DF0538FFC22901A0D74A5F102901A0E3A
:10173700745AF102227A3079D07820901A40D1FD7C
:10174700E520F709A3DAF7227A3079D0901A40E733
:10175700F10209A3DAF922AB74A875BB01027980FB
:10176700BB02027981BB03027982BB04027994BB75
:1017770005027983BB06027986BB07027992BB080B
:10178700027987BB0902799CBB0A027988BB0B02E5
:101797007989E8F7227C05120562DCFB22C2AF12C9
:1017A7000572120579120580120587120553120575
:1017B70072120579120580120587120553120572F8
:1017C700120579120580120587D2AF22C2AF120522
:1017D70087120580120579120572120553120587C3
:1017E7001205801205791205721205531205871228
:1017F7000580120579120572D2AF22AE74AF75C299
:10180700AF120572120572120572120553DEF2123B
:101817000587120553DFF8D2AF221217A412179CBF
:1018270012179C75740175750175760011027C0598
:10183700AD5C120562C3ED955C70F5C3E55C940180
:10184700400AC3E55C94FF403702186412175E1222
:1018570016BB1217A4C2AF75EF1212179CDCD10585
:0F18670076C3E5769403500280C212179C057574
:10187600E5741490009F93F808C3E57598500280AC
:10188600A912179C12179C0574C3E574940C500298
:101896008095120FE41216BBC2AF75EF1212179C99
:0319FD0002115E76
:101A00000E061507070104FFFF09020101A55A018F
:101A100000B4FFFFFF03FF01FF25D078C804FF01DA
:091A200000FF0A010100FF00FFB4
:101A4000235467794B463430412320202020202026
:101A500023424C48454C4923463331302320202033
:101A60002020202020202020202020202020202076
:101C0000C2AFC2D353D9BF7581C043B20343FF8073
:101C1000752438752503B1C975EF0275E24043F1AB
:101C20002053A4DF75D4FFD2857DFA780379E67C52
:101C300010752200752300901DD67B0675249875BB
:101C400025013085028142208508D8FBD9F9DCF7CF
:101C500081B4308508D8FBD9F9DCF781B4B189E4C7
:101C600093A3C39A6004DDC381B4DBDBB17B600264
:101C7000812B7B08E493FAA3B15CDBF87A30B15C8A
:101C8000752200752300B17BEAFCEBFDC3ED94FEE9
:101C9000400EB17B8A278B28ED30E0048A828B834B
:101CA000B17B7AC270D8C3ED94FE601350CEBD00F4
:101CB00025EC60097520007521FF0200008100A855
:101CC00027A9280809D804D90281D3B17FEA89AAB3
:101CD000F281C50D81A0C3ED94035049EDA2E092BD
:101CE000007AC5C3E5829400E583941C50902000DF
:101CF00010438F02438F0175B7A575B7F1F030001F
:101D00001FA827A9280809438F01538FFDD804D99C
:101D100002A12089AAE275B7A575B7F1F0A3A10DBC
:101D2000538FFC817C7AC1BD030CE493A3FAB140CC
:101D3000DCF8B138817C817EAA22AB23B15CEBFA5E
:101D4000EA6222752608C3E52313F523E52213F57D
:101D50002250066323A0632201D526EAB1C9B1C986
:101D600075260AEAF4200102D285300102C285B14B
:101D7000C9C3134002C201D526EB22B17FEAFB2082
:101D80008502A17F308502A184752608AE24AF2587
:101D9000C3EF13FFEE13FEB1CDB1C9C3EA13308513
:101DA000024480FA30E703632201C3E52313F523DD
:101DB000E52213F52250066323A0632201D526D91C
:101DC000E52265236523F52222AE24AF250E0FDE22
:101DD000FEDFFCD20122424C48656C693437316326
:041DE000F3100601F5
:00000001FF
